:100000000C94AA000C9420020C94C7000C94C70016
:100010000C94C7000C94C7000C94C7000C94C70044
:100020000C94C7000C94C7000C94C7000C94C70034
:100030000C94C7000C94C7000C94C7000C94C70024
:100040000C94C7000C94C7000C94C7000C94C70014
:100050000C94C7000C94C7000C94C7000C94C70004
:100060000C94C7000C94C700180372006100700064
:1000700068006E00650074002E006E00650074005C
:10008000040309040A033100300030003000050188
:100090000904A1010901A1008501093009311500F8
:1000A00026FF007508950281020509190129081526
:1000B000002501750195088102C0C005010904A150
:1000C000010901A100850209300931150026FF0050
:1000D00075089502810205091901290815002501F5
:1000E000750195088102C0C005010904A10109013B
:1000F000A100850309300931150026FF0075089518
:1001000002810205091901290815002501750195CB
:10011000088102C0C005010904A1010901A10085EF
:100120000409300931150026FF0075089502810287
:100130000509190129081500250175019508810295
:10014000C0C012010101000000089B280300040147
:100150000102030111241FBECFEFD4E0DEBFCDBFEB
:1001600011E0A0E0B1E0ECE4FEE002C005900D92E9
:10017000AC34B107D9F721E0ACE4B1E001C01D9285
:10018000AB3AB207E1F70E9445060C9424070C94A1
:100190000000CF93C62F2091000124FF0BC02091B7
:1001A000810138E8232720938101FC01A2E8B1E016
:1001B0008C2F04C02AE520930001F7CF815018F05E
:1001C00091919D93FBCF6C2F82E891E00E941C02DD
:1001D000CC5FC0930001CF910895CF93DF938091BE
:1001E000910118160CF0AEC090918E0120918D01F6
:1001F0002D3219F090E880E09FC02AE5209301019C
:100200008B30C1F7CCE0D0E0C91BD109CB56DE4F13
:100210008881807609F080C010927F0189818111E8
:100220000BC0109280018FE791E090939001809332
:100230008F0190E882E079C0853021F48A81809333
:10024000920171C0863009F04BC08B81813009F476
:1002500042C0823021F4CE010E94830360C083300B
:1002600069F58A81811109C080E890E0909390013E
:1002700080938F0190EC84E058C0813049F488E687
:1002800090E09093900180938F0190EC88E14DC0B5
:10029000823049F485E291E09093900180938F0140
:1002A00090E886E142C08330E1F584E890E09093E5
:1002B000900180938F0190EC8CE037C0813249F43B
:1002C0008FE591E09093900180938F0190EC89E00D
:1002D0002CC0823231F5CE010E94830390EC25C000
:1002E000883019F484E991E00AC0893021F48A81C8
:1002F0008093940118C08A3049F48FE791E090937D
:10030000900180938F0190E881E00FC08B3059F409
:1003100083EC8093810107C0CE010E94B10390E875
:1003200004C090EC01C090E880E02F81211104C04E
:100330002E81281708F4822F90934C01809302019C
:10034000109291018091010184FF46C080910201C9
:100350008F3F09F441C0C82F893008F0C8E08C1BDA
:100360008093020120914C0120FD02C0DBE401C01A
:10037000D3EC2F5F20934C0180918F0190919001DD
:1003800026FD05C0FC01A7E7B1E02C2F0AC0A7E7B6
:10039000B1E0FC012C2F215048F034913D9331966F
:1003A000FACF215018F031913D93FBCF8C0F911D66
:1003B0009093900180938F016C2F87E791E00E94CA
:1003C0001C0284E08C0FC83019F09FEF909302015B
:1003D000D0937601809301018AE099B1957031F450
:1003E0008150D9F71092920110928C01DF91CF9138
:1003F0000895E9E6F0E0808183608083E89A83ECE9
:10040000809381010895A82FB92F8FEF9FEF41E0CE
:1004100050EA615070F02D9138E0722F7827969550
:100420008795269570FF02C0842795273A95A9F7EE
:10043000F0CF809590950895E6DF8D939D93089574
:10044000CF93CFB7CF93489BFECF489B09C0489B23
:1004500007C0489B05C0489B03C0489B01C09EC085
:10046000DF93C0918E01DD27CB56DE4F489B02C043
:10047000DF91EBCF2F930F931F9309B12FEF00FB69
:1004800020F94F933F9319B14FEF012700FB21F95A
:100490003BE031C04E7F012F19B1216028C0102FE1
:1004A0004D7F2260000009B129C04B7F2460012FDD
:1004B000000019B12BC019B1477F28602AC04F7EB8
:1004C00009B120612CC04F7D19B120622FC04F7B34
:1004D00009B1206432C0422709B149934FEF0000AF
:1004E000102710FB20F919B11570A9F1297F91F29D
:1004F000012700FB21F909B1237F89F23150F0F186
:10050000102710FB22F919B1277E79F2012700FB91
:1005100023F92F7C81F209B1102710FB24F92F79E0
:1005200071F200C019B1012700FB25F92F7359F2B0
:1005300000C009B1102710FB26F9223040F200C09C
:1005400019B1012700FB27F9243028F64F772068DE
:1005500019B10000F9CF3B503195333011E01CBB8D
:10056000B8F0C31BD0400881033C41F10B3431F19A
:100570001981412F1F7720918C01121731F4093610
:1005800091F10D3279F0013E69F022272093930119
:100590003F914F911F910F912F91DF91CF91CFBF3D
:1005A000CF911895009393013F914F911F910F9117
:1005B0002F91DF91CCB3C0FD46CFF0CF00919301D6
:1005C000002331F3109191011123A1F53430A2F1F0
:1005D0003093910100938D0110918E013BE0311B0E
:1005E00030938E0129C00091910101301CF50AE57C
:1005F00047FD09C03091010134FD20C00093010185
:10060000C6E7D1E01FC03091000134FD17C0009350
:100610000001C1E8D1E016C0052710E00BB91FC0EA
:10062000052722C0052727C005272CC0052710E075
:100630000BB933C04AE503C042ED01C0432FC4E10A
:10064000D0E032E01AB11560589A0BB11AB95F9335
:1006500055E020E820FF05270BB9279517951C3F8B
:10066000D8F620FF052727950BB917951C3FC0F634
:1006700020FF0527279517950BB91C3F98F620FFFB
:100680000527279517951C3F0BB970F600C04991B7
:1006900020FF05270BB9279517951C3F38F620FF3B
:1006A000052727950BB917951C3F38F520FF05271F
:1006B000279517950BB91C3F10F520FF05272795A7
:1006C00017951C3F0BB9E8F4242F3A9519F60A7FC9
:1006D0005F910BB900C010919201C651D04011F04A
:1006E00010938C0111E01CBB01601AB11A7F402FDE
:1006F0004A7F0BB91AB94BB94BCF0527D3CF052782
:10070000D8CF0527DDCFFC018081807641F591812E
:10071000963031F593819230D1F0923269F0913078
:10072000F9F480915E0190915F0190939001809324
:100730008F0180915D010895809161019091620126
:100740009093900180938F0180916001089583E0E0
:1007500091E09093900180938F0182E2089580E070
:100760000895DC018FE491E09093900180938F01D4
:100770008C918076803299F411968C91119781300A
:1007800071F410924E01E0915B01F0915C010784DD
:10079000F089E02D12966C918FE491E0099480E04D
:1007A000089581502091640190E0222369F0DC01DA
:1007B000A259BE4FFC01EA59FE4F81E02C91908175
:1007C00029130DC080E00895880F991FBC016A5954
:1007D0007E4F42E050E082599E4F0E9417070895D5
:1007E00080916401882309F445C0449A20E32A9546
:1007F000F1F7449888E090E040E050E068E16A95C5
:10080000F1F74598550F440F339B5160329B41607F
:1008100028E12A95F1F7459A0197009779F788E042
:1008200090E020E030E068E16A95F1F74598330FF9
:10083000220F339B3160329B216068E16A95F1F7AA
:10084000459A0197009779F788E090E068E16A950A
:10085000F1F7459868E16A95F1F7459A0197009795
:10086000A9F750936E0140936F013093700120936C
:100870007101089580916301449A882309F468C046
:1008800080E38A95F1F7449820E32A95F1F72D9AB1
:1008900068E16A95F1F788E090E040E050E0459823
:1008A00028E12A95F1F7550F440F339B5160329B95
:1008B0004160459A68E16A95F1F70197009779F7E9
:1008C00050936E014093700188E090E0459828E1D4
:1008D0002A95F1F756954695339B5068329B4068B0
:1008E000459A68E16A95F1F70197009779F72D9895
:1008F00088E18A95F1F788E090E020E030E04598C3
:1009000068E16A95F1F7330F220F339B3160329B18
:100910002160459A68E16A95F1F70197009779F7A8
:10092000309372012093740188E090E0459868E16B
:100930006A95F1F736952695339B3068329B20688F
:10094000459A68E16A95F1F70197009779F742C0F7
:1009500080E38A95F1F7449888E090E020E030E069
:1009600040E050E068E16A95F1F74598550F440F73
:10097000330F220F339B5160329B4160319B3160BA
:10098000309B216068E16A95F1F7459A01970097DD
:1009900049F750936E014093700130937201209398
:1009A000740188E090E068E16A95F1F74598569502
:1009B000469536952695339B5068329B4068319B0F
:1009C0003068309B206868E16A95F1F7459A019795
:1009D000009749F780914A01882321F180916501B0
:1009E0005F3F11F4816001C08E7F8093650180912B
:1009F00065014F3F11F4826001C08D7F80936501D6
:100A0000809165013F3F11F4846001C08B7F80932A
:100A10006501809165012F3F11F4886001C0877FD7
:100A2000809365018091650180FD50E050936F01D6
:100A300081FD40E04093710182FD30E0309373010D
:100A400083FD20E0209375010895CF93CFB7F894EC
:100A50003C9A3D9A87B1807F87B988B18F6088B909
:100A6000459A4498259A2D9A109265010E94F003A8
:100A700080914A01811124C080916F018F3F29F438
:100A800080916501816080936501809171018F3F44
:100A900029F48091650182608093650180917301E2
:100AA0008F3F29F480916501846080936501809176
:100AB00075018F3F29F480916501886080936501FD
:100AC000449A40E34A95F1F7449830E020E080E012
:100AD00090E048E14A95F1F74598339905C0833194
:100AE000910519F431E001C02F5F48E14A95F1F713
:100AF000459A01968831910561F7332329F0273112
:100B000019F481E0809364012D98329B0FC0449AC0
:100B100080E38A95F1F7329909C0449840E34A95F9
:100B2000F1F7329B03C081E0809363012D9A329BE1
:100B30000FC0449A80E38A95F1F7329909C044982E
:100B400040E34A95F1F7329B03C081E08093630153
:100B5000CFBFCF910895FC01653008F085C080912A
:100B60006401462F552747FD509541505109882370
:100B700009F1DA01A259BE4F3097B1F060839C9120
:100B800090FD02C080E801C08FEF91FD80E081837D
:100B90009C9192FD02C080E801C08FEF93FD80E040
:100BA00082838C91807F8383FA01EA59FE4F8C9176
:100BB000808358C0CA01880F991F309709F448C034
:100BC0006083DC01A259BE4F3C9130FD02C020E899
:100BD00001C02FEF31FD20E021833C9132FD02C0A6
:100BE00020E801C02FEF33FD20E022832091650132
:100BF00030E002C0359527954A95E2F720FF04C002
:100C00002C91207F238324C02C91622F661F66279E
:100C1000661F11964C9130E1439FA0011124642B73
:100C2000422F407450E035E0559547953A95E1F7ED
:100C3000642B422F407250E073E0559547957A95AA
:100C4000E1F7642B207130E035952795622B6383A3
:100C5000FC01EA59FE4FDC01A259BE4F8D919C91D7
:100C60009183808384E0089580E0089510924A0182
:100C700008958EE890E090933D0180933C0189E3D4
:100C800091E0089582E190E0089581E084B98EEFCB
:100C900085B917B88FEF88B988EF8BB985E08AB925
:100CA00082E08093B00087E08093B10084EC809371
:100CB000B3008FE295E70197F1F700C0000083B120
:100CC0008670843011F40E9436060E943906FC01B9
:100CD00090935C0180935B01838194819093620186
:100CE0008093610181818093600187819085009765
:100CF00031F090935F0180935E01858108C082E4AA
:100D000091E090935F0180935E010E944206809380
:100D10005D018091600180931C018BB18A7F8BB94A
:100D20008AB185608AB987EC9FEA0197F1F700C024
:100D300000008AB18A7F8AB9E0915B01F0915C0181
:100D40000184F285E02D09950E94F901E0915B0193
:100D5000F0915C010384F485E02D0995789482E09C
:100D6000D82E01E010E0A8950E94ED00B99BFBCFC2
:100D7000D7BAE0915B01F0915C010384F485E02D2A
:100D80000995C0E0D0E0E12CE0915B01F0915C01BD
:100D90008081992787FD9095C817D9078CF4058421
:100DA000F685E02D8C2F8F5F0995882339F0C801D7
:100DB0000C2E01C0880F0A94EAF7E82A2196E4CFA6
:100DC000EE2089F2C0E0D0E0FF24E7FCF094E0914F
:100DD0005B01F0915C018081992787FD9095C81790
:100DE000D9070CF0C0CFC7010C2E02C0959587958E
:100DF0000A94E2F780FF19C08091000184FF15C0BA
:100E00000784F089E02D6C2F6F5F8FE491E00995E6
:100E1000682F8FE491E00E94C9008091000184FD59
:100E200004C00E94ED00A895F8CF2196D0CFFB0119
:100E3000DC0104C08D910190801921F44150504093
:0C0E4000C8F7881B990B0895F894FFCFA9
:100E4C005A5AFF09022200010100803209040000F5
:100E5C000103000000092101010001220000070527
:100E6C00810308000A140334006E0065007300341B
:100E7C000073006E006500730004B40000000000F5
:0C0E8C0000002505F003D103AB050100B8
:00000001FF
